:1000000012C0D6C418951895189518951895189576
:100010001895189518951895189518951895189578
:100020001895189518958FE58DBFC0EEE8EF4E2E08
:1000300084E08EBFD3E0F2E05F2EEEEFF3E0A0E6C7
:10004000B0E088278D933197E9F7F4D96624889A30
:1000500078948BB780648BBF85B78C7F85BFBB9A44
:10006000BC9ABD9A889889988A988B988C988D9A12
:100070008E9A8F98909A919A929A939A949A979A24
:10008000BFD9EEE0FFE1B6D98FEB11E0C8D9E0E2CD
:10009000FFE1B0D9E2E0F0E0C4D9A6E6B0E080B379
:1000A0008C93A6E6B0E08C9183718C938AEA80935E
:1000B000600081E08093DF0084E08093850085E02C
:1000C0008093860086E08093870087E08093880095
:1000D00089E0809389008BE080938A00A3EAB0E0F6
:1000E000E2EBFEE13BDDA7EAB0E0E6EBFEE136DD68
:1000F000ABEAB0E0EAEBFEE131DDAFEAB0E0EEEB17
:10010000FEE12CDDA3EBB0E0E2ECFEE127DDA7EBA6
:10011000B0E0E6ECFEE122DDACEBB0E0E2E3FFE1D3
:10012000FADAA1ECB0E0E8E3FFE1F5DAA6ECB0E042
:10013000EEE3FFE1F0DAABECB0E0E4E4FFE1EBDAB0
:10014000A0EDB0E0EAE4FFE1E6DAA5EDB0E0E0E53D
:10015000FFE1E1DAA8E0B1E0E6E5FFE1DCDAACE0FE
:10016000B1E0EAE5FFE1D7DAA0E1B1E0EEE5FFE1D9
:10017000D2DAA4E1B1E0E2E6FFE1CDDAA9E1B1E053
:10018000E6E6FFE1C8DAADE1B1E0EAE6FFE1C3DAB5
:10019000A2E2B1E0EEE6FFE1BEDAA5E2B1E0E2E71D
:1001A000FFE1B9DAA8E2B1E0E6E7FFE1B4DAABE2F9
:1001B000B1E0EAE7FFE1AFDAAEE2B1E0EEE7FFE19E
:1001C000AADA81E08093310181E08093210181E00E
:1001D0008093180183E08093BB00A2E6B0E0E0E0EA
:1001E000F0E094E0AFDD849914C0EAECFEE18ADC33
:1001F000E9E0F0E0ADE0BB2794E07BE792DDEEECD8
:10020000FEE180DCE5E0F0E0ADE0BB2794E07BE7D9
:1002100088DDA3E0B1E0E5E0F0E094E093DDA5E760
:10022000B0E0E9E0F0E094E08DDDE4E0F0E0A7E0AC
:10023000B1E085DD00916600003109F001C0F3D521
:100240008CE040D9DDD8E2E8FFE1D4D85A924A9256
:10025000E2E6F0E0A42DB52D4DDD84E091D804D880
:10026000229684E089D88FEB11E0D9D8E8E8FFE145
:10027000C1D8A0EEB0E0B8D8E2E0F0E0D2D85A920F
:100280004A92E3E0F1E0A42DB52D34DD84E078D886
:10029000EBD7229684E070D8B3D8EEE8FFE1AAD875
:1002A000A0EEB0E0A1D88FEB11E0B9D8E6E9FFE10C
:1002B000A1D8A0EEB2E0E7E0F1E0CADC93D8E2E03A
:1002C000F0E0AFD89DD8A8E1B1E00D91112744E04E
:1002D00050E017DAA4E0B1E0A00FB11F85D8EEE935
:1002E000FFE188D8A1E2B1E00D91112744E050E090
:1002F00008DAA5E1B1E0A00FB11F76D85A924A9270
:10030000E5E7F0E0A42DB52DF5DC84E039D8FAD787
:10031000229684E031D89BD38FEB1DE080D8ABEBE5
:10032000B0E00D91112745E050E0EBD9A7EBB0E02C
:10033000A00FB11F59D88FE71FE071D8A0EEB2E02F
:10034000E7E0F1E085DC4ED8E5E7F0E0A2E3B1E0DC
:10035000D1DCA6E3B1E0EEECFEE100DCBB27A0E3DC
:100360000C9107FB81E00EF480E08F93A1E6B0E0F2
:100370008C9184FB81E00EF480E09F918923882397
:1003800009F41DC0E5E7F0E0A1E7B0E0B3DCE2E38B
:10039000F1E0A5E7B0E0AEDC809161008061809380
:1003A00061005A924A92E5E7F0E0A42DB52DA2DC57
:1003B00084E0E6D7A7D7229684E0DED748D3BB27D0
:1003C000A0E30C9107FB81E00EF080E08F93A1E6A3
:1003D000B0E08C9184FB81E00EF080E09F91892356
:1003E000882309F418C0E1E7F0E0A5E7B0E082DC7B
:1003F000809161008F7E809361005A924A92E5E776
:10040000F0E0A42DB52D76DC84E0BAD77BD7229618
:1004100084E0B2D71CD3E5E7F0E01CDAE2EDFEE1C0
:100420007ADB82DB08F004C0C398C498C59A8AC0FE
:10043000E5E7F0E00FDAE2EDFEE16DDB75DB81E090
:1004400008F480E08F93E5E7F0E004DAE6EDFEE102
:1004500062DB6ADB81E010F009F080E09F91892384
:10046000882309F404C0C398C49AC5986BC0E5E713
:10047000F0E0F0D9E6EDFEE14EDB56DB81E008F47A
:1004800080E08F93E5E7F0E0E5D9EAEDFEE143DBBC
:100490004BDB81E010F009F080E09F9189238823F5
:1004A00009F404C0C398C498C5984CC0E5E7F0E0CF
:1004B000D1D9EAEDFEE12FDB37DB81E008F480E003
:1004C0008F93E5E7F0E0C6D9EEEDFEE124DB2CDB0F
:1004D00081E010F009F080E09F918923882309F4DE
:1004E00004C0C39AC49AC59A2DC0E5E7F0E0B2D91A
:1004F000EEEDFEE110DB18DB81E008F480E08F9385
:10050000E5E7F0E0A7D9E2EEFEE105DB0DDB81E0F7
:1005100010F009F080E09F918923882309F404C03A
:10052000C39AC498C59A0EC0E5E7F0E093D9E2EE0D
:10053000FEE1F1DAF9DA10F009F001C003C0C39866
:10054000C49AC59AA6E6B0E080B38C93A6E6B0E064
:100550008C9183718C9300916600033109F4B5C1CD
:1005600084E190E0E0D7A6E6B0E080B38C93A6E605
:10057000B0E08C9183718C9300916600003109F09A
:100580002FC0A8E1B1E08C918F5F8C93009118018E
:10059000043010F009F001C003C081E0809318011D
:1005A00000911801013009F003C0959A969A11C084
:1005B000023009F003C0959A96980BC0033009F0F9
:1005C00003C09598969A05C0043009F002C095982A
:1005D00096988FE71CE023D7E4EAFFE10BD742C1EE
:1005E000023109F037C0A1E2B1E08C918F5F8C93AA
:1005F00000912101023010F009F001C003C081E038
:10060000809321018FE71CE00AD7E4EAFFE1F2D6EC
:1006100000912101013009F006C0E2E3F1E0A5E715
:10062000B0E068DB08C0023009F005C0E5E7F0E0A3
:10063000A2E3B1E05FDB5A924A92E5E7F0E0A42D35
:10064000B52D58DB84E09CD65DD6229684E094D606
:10065000FED108C1013109F05AC0A1E3B1E08C918B
:100660008F5F8C9300913101043010F009F001C0CC
:1006700003C081E0809331018091610080628093AA
:1006800061008FE71CE0CBD6A1E3B1E00D9111270B
:1006900043E050E036D8AFE1B1E0A00FB11FA4D6DF
:1006A00000913101013009F007C0A1E8B0E0E9E0B4
:1006B000F0E094E047DB1DC0023009F007C0A1E87C
:1006C000B0E0EDE0F0E094E03DDB13C0033009F072
:1006D00007C0A1E8B0E0E1E1F0E094E033DB09C05D
:1006E000043009F006C0A1E8B0E0E5E1F0E094E0F4
:1006F00029DB5A924A92E1E8F0E0A42DB52DFADA0E
:1007000084E03ED6FFD5229684E036D6ABC00330D7
:1007100009F04FC0A1E6B0E08C9185FB0EF02EC031
:1007200000913101013009F008C0E9E0F0E0A5E7EF
:10073000B0E094E07BE7F5DA20C0023009F008C0B1
:10074000EDE0F0E0A5E7B0E094E07BE7EADA15C081
:10075000033009F008C0E1E1F0E0A5E7B0E094E083
:100760007BE7DFDA0AC0043009F007C0E5E1F0E01A
:10077000A5E7B0E094E07BE7D4DA0FC0ABEBB0E0E4
:100780008C918F5F8C930091BB00063010F009F0C4
:1007900001C003C081E08093BB00809161008F7D28
:1007A000809361008FE71CE03AD6E4EAFFE122D6AD
:1007B00059C0013009F056C0A1E6B0E08C9185FB2C
:1007C0000EF038C000913101013009F007C0A5E7F3
:1007D000B0E0E9E0F0E094E0B5DA1DC0023009F0E5
:1007E00007C0A5E7B0E0EDE0F0E094E0ABDA13C0BD
:1007F000033009F007C0A5E7B0E0E1E1F0E094E0E4
:10080000A1DA09C0043009F006C0A5E7B0E0E5E1CF
:10081000F0E094E097DA5A924A92E5E7F0E0A42DEE
:10082000B52D68DA84E0ACD56DD5229684E0A4D5E8
:100830000ED10DC08091BB0081508093BB00009110
:10084000BB00013008F003C086E08093BB008091BC
:1008500061008F7D809361008FE71CE0E0D5E4EAC2
:10086000FFE1C8D58FE711E0DAD5A8E1B1E00D913D
:10087000112744E050E045D7A4E0B1E0A00FB11F3C
:10088000B3D58FEB1DE0CBD5ABEBB0E00D911127CD
:1008900045E050E036D7A7EBB0E0A00FB11FA4D5DC
:1008A0008FE715E0BCD5E8EAFFE1A4D5A1E2B1E00D
:1008B0000D91112744E050E024D7A5E1B1E0A00F4D
:1008C000B11F92D58CE291E02ED6A1E6B0E08C91DA
:1008D00087FB0EF06AC0809161008F778093610082
:1008E000A1E6B0E08C9186FB0EF027C0EBEBF0E0C8
:1008F000A190BB24EFE9F0E0AA0CBB1CAA0CBB1C26
:10090000EA0DFB1DACD7E5E7F0E0A4D7A9D8FF2797
:10091000EDE0A5E7B0E0EED9E5E7F0E09BD7E6EE45
:10092000FEE1F9D801D910F009F001C005C0A5E732
:10093000B0E0E6EEFEE112D924C0EBEBF0E0A190CE
:10094000BB24EFE9F0E0AA0CBB1CAA0CBB1CEA0D0F
:10095000FB1D85D7E5E7F0E07DD773D8FF27EDE0F5
:10096000A5E7B0E0C7D9E5E7F0E074D7EAEEFEE12D
:10097000D2D8DAD808F005C0A5E7B0E0EAEEFEE18B
:10098000EDD88FE711E04BD55A924A92E5E7F0E0B7
:10099000A42DB52DAFD984E0F3D4B4D4229684E04D
:1009A000EBD455D08BB780648BBFD8CCF894FFCFF5
:1009B0000F921F922F923F924F925F927F92AF922F
:1009C000BF920F931F932F933F934F935F936F9318
:1009D0007F938F939F93AF93BF93CF93DF93EF93C7
:1009E000FF938FB78F938BB78F7B8BBF82E090E0A5
:1009F0009AD580916100806880936100839906C0D8
:100A0000809161008F7B8093610005C080916100BF
:100A10008064809361008F918FBFFF91EF91DF9190
:100A2000CF91BF91AF919F918F917F916F915F9186
:100A30004F913F912F911F910F91BF90AF907F9059
:100A40005F904F903F902F901F900F901895A9E7BF
:100A5000B0E0EEEEFEE182D881E08093DA00009112
:100A6000DA00063010F009F074C0E5E7F0E0F7D6E0
:100A7000EAEDF0E0A190BB24E4E8F0E0EA0DFB1D14
:100A8000D080EE24FF24002709D7AAD7FF27EDE066
:100A9000A9E6B0E02FD982E090E0ABEDB0E08D9315
:100AA0009C93ABEDB0E00D911C91003850E0150720
:100AB00010F009F047C0EBEDF0E0D190E080FF24AA
:100AC0000027ECD61CD7E9E6F0E0C4D689D7FF278B
:100AD000EDE0A9E7B0E00ED9E9E7F0E0BBD6E2EF40
:100AE000FEE119D821D810F009F001C01DC0E9E7D6
:100AF000F0E0B0D6EEEEFEE10ED816D808F014C045
:100B0000AAEDB0E0AD90BB24A4E8B0E0AA0DBB1DF7
:100B10008C918093DF00ABEDB0E08D919C91ADEDB9
:100B2000B0E08D939C9315C0ABEDB0E00D911C919E
:100B300042E050E0040F151FABEDB0E00D931C93A5
:100B400008F0AFCFAAEDB0E08C918F5F8C9308F4E2
:100B500086CFE2E6F0E083D6E9E7F0E07BD6EAD69E
:100B6000FF27EDE0ADE6B0E0C5D8AFEDB0E08C9189
:100B700084508C938091DF0080938B0095E0ABE8EC
:100B8000B0E0CED50091DD0041E0041BACE8B0E060
:100B90000C9392E0ACE8B0E0CBD500918B00409193
:100BA0008C00042BABE8B0E00C930091DD0041E039
:100BB000041BACE8B0E00C9396E0ACE8B0E0B0D534
:100BC000EDE6F0E0EED8FF27EDE006D6A5E9B0E0CF
:100BD000DD92EC92EDE6F0E0C5D8FF27EDE0A7E965
:100BE000B0E088D89CE1E7E9F0E015D9FF27EDE017
:100BF000A7E9B0E07FD8E7E9F0E0D3D8FF27EDE040
:100C0000EBD5ABE9B0E0EDE0FF2774D8009195009B
:100C10004FE00423ADE8B0E00C9394E0ADE8B0E021
:100C20007FD594E0A5E9B0E08BD5A5E9B0E00D91C2
:100C30001C914FE350E004231523A5E9B0E00D9388
:100C40001C9300918C0040919500040FACE8B0E03B
:100C50000C93ABE9B0E00D911D912D913C9140E0DA
:100C600050E060E07FE04ED4AFE9B0E00D931D931B
:100C70002D933D9398E1AFE9B0E06DD500918D00E3
:100C800040919F00040FADE8B0E00C93ABE9B0E0F9
:100C90000D911D912D913C9140E050E06FEF70E07F
:100CA00031D4AFE9B0E00D931D932D933D9390E1C6
:100CB000AFE9B0E050D580919F0080938E00ABE902
:100CC000B0E00D911D912D913C9140E05FEF60E00F
:100CD00070E018D4AFE9B0E00D931D932D933D93D0
:100CE00098E0AFE9B0E037D580919F0080938F0006
:100CF000ABE9B0E00D911D912D913C914FEF50E08B
:100D000060E070E0FFD3AFE9B0E00D931D932D9349
:100D10003D9380919F0080939000E6E3F1E09FD5A2
:100D2000E9E7F0E097D58DD6FF27EDE0ADE6B0E03E
:100D3000E1D7EDE6F0E013D8FF27EDE0ADE6B0E057
:100D4000D9D7EDE6F0E086D5E6EFFEE1E4D6ECD6C5
:100D500010F009F001C00CC0E9E7F0E0A6E3B1E053
:100D6000C9D780E290E0ADEDB0E08D939C9306C0D2
:100D700080E190E0ADEDB0E08D939C9366D8A0E665
:100D8000B0E01C9179D819E877D8ADEDB0E01C91AE
:100D900073D869D887E090E0ABEDB0E08D939C9379
:100DA000ABEDB0E00D911C910C3050E0150710F048
:100DB00009F019C04AD8A0E6B0E01C915DD8ABEDAF
:100DC000B0E01C9159D8ABEDB0E0AD90BC90A4E878
:100DD000B0E0AA0DBB1D1C914FD845D8ABEDB0E0DB
:100DE000D3D208F0DDCF31D8A0E6B0E01C9144D8D2
:100DF00019E842D810E040D836D8EDE6F0E02AD520
:100E0000EAEFFEE188D690D610F009F001C00AC0E2
:100E10001CD8A0E6B0E01C912FD817E82DD810E41C
:100E20002BD821D80895A5E7B0E0EAECFEE196D6EC
:100E300081E080933A01E4D2E2E8FFE1DBD28FEB7C
:100E400011E0EDD2EEEAFFE1D5D2E1E0F0E0E9D247
:100E5000A6E6B0E080B38C93A6E6B0E08C918371F7
:100E60008C9300916600033109F480C00091660004
:100E7000003109F015C0AAE3B1E08C918F5F8C932B
:100E800000913A01033010F009F001C003C081E085
:100E900080933A018091610088608093610063C013
:100EA000023109F013C080913A01815080933A01D8
:100EB00000913A01013008F003C083E080933A01C9
:100EC000809161008860809361004DC0013109F01C
:100ED0001DC096D2E6EBFFE18DD2E0E0F0E0A2E6A5
:100EE000B0E094E07BE71DD7E4E0F0E0A7E0B1E0FC
:100EF0007BE714D7E5E0F0E0A3E0B1E094E07BE726
:100F000010D7E1E0F0E08DD2AEC12DC0033009F082
:100F100015C0ABEBB0E08C918F5F8C930091BB0060
:100F2000063010F009F001C003C081E08093BB00DF
:100F30008091610088608093610015C0013009F0E4
:100F400012C08091BB0081508093BB000091BB0018
:100F5000013008F003C086E08093BB0080916100FF
:100F60008860809361008CE291E0DDD2A1E6B0E080
:100F70008C9187FB81E00EF080E08F93A1E6B0E0DA
:100F80008C9183FB81E00EF080E09F91892B882378
:100F900009F44EC100913A01013009F083C0A1E685
:100FA000B0E08C9187FB0EF059C0A1E6B0E08C91C7
:100FB00086FB0EF027C0EBEBF0E0A190BB24EFE93D
:100FC000F0E0AA0CBB1CAA0CBB1CEA0DFB1D47D40D
:100FD000E2E6F0E03FD444D5FF27EDE0A2E6B0E042
:100FE00089D6E2E6F0E036D4EEEFFEE194D59CD56A
:100FF00010F009F001C005C0A2E6B0E0EEEFFEE19E
:10100000ADD524C0EBEBF0E0A190BB24EFE9F0E01C
:10101000AA0CBB1CAA0CBB1CEA0DFB1D20D4E2E6EB
:10102000F0E018D40ED5FF27EDE0A2E6B0E062D6DE
:10103000E2E6F0E00FD4E2E0FFE16DD575D508F00F
:1010400005C0A2E6B0E0E2E0FFE188D58091610052
:101050008F77809361008BB780648BBF5A924A92DE
:10106000E2E6F0E0A42DB52D45D684E089D1FCD090
:10107000229684E081D1C4D1ECEBFFE1BBD18FEBB0
:1010800011E0CDD1E8ECFFE1B5D18FEB11E0C7D194
:10109000A0EEB0E0A9D1DBDC809161008860809394
:1010A0006100C6C0023009F077C0A1E6B0E08C91C3
:1010B00087FB0EF054C0A1E6B0E08C9186FB0EF0E9
:1010C00017C0EBEBF0E0A190BB24EFE9F0E0AA0C35
:1010D000BB1CAA0CBB1CEA0DFB1DC1D3E3E0F1E075
:1010E000B9D3BED4FF27EDE0A3E0B1E003D62FC013
:1010F000EBEBF0E0A190BB24EFE9F0E0AA0CBB1C05
:10110000AA0CBB1CEA0DFB1DAAD3E3E0F1E0A2D3BD
:1011100098D4FF27EDE0A3E0B1E0ECD5E3E0F1E007
:1011200099D3E6E0FFE1F7D4FFD408F010C0E3E084
:10113000F1E090D3EAE0FFE1EED4F6D410F009F04C
:1011400001C005C0A3E0B1E0EEECFEE107D580915F
:1011500061008F77809361008BB780648BBF5A9258
:101160004A92E3E0F1E0A42DB52DC4D584E008D186
:101170007BD0229684E000D143D1E4EDFFE13AD167
:101180008FEB11E04CD1A0EEB0E02ED18091610048
:101190008860809361004CC0033009F049C0A1E62B
:1011A000B0E08C9187FB0EF02BC0A1E6B0E08C91F3
:1011B00086FB0EF010C0A7E0B1E08C918F5F8C939E
:1011C00000910701043610F009F001C003C084E665
:1011D000809307010DC08091070181508093070122
:1011E00000910701013008F003C081E080930701FE
:1011F000809161008F77809361008BB780648BBF93
:10120000FFD0ECEDFFE1F6D08FEB11E008D1E6E97D
:10121000FFE1F0D0A0EEB2E0E7E0F1E019D5E2D0D6
:10122000E2EEFFE1E7D08091610088608093610089
:10123000A1E6B0E08C9183FB0EF014C08FEB1DE0B3
:10124000EED0ABEBB0E00D91112745E050E059D264
:10125000A7EBB0E0A00FB11FC7D080916100877FDE
:1012600080936100F5CD0895A0EEB2E0AF93BF93F7
:10127000E881F981EFD266D111E005E0BF91AF912D
:1012800082D4E0EEF2E0A0EEB0E02FD5A0EEB0E028
:10129000E8EEFFE12FEF91E074D2A1E0B1E00C9312
:1012A0000091010143E0040FA2E0B1E00C93E0EEF5
:1012B000F0E000910201ABEEB0E022D50091010117
:1012C00044E0040FA2E0B1E00C93A0EEB0E041D501
:1012D000EA2FFB2F3397F0400FEFA6EFB0E010D5C9
:1012E000EBEEF0E0A0EEB0E000D5A0EEB0E073D001
:1012F000E8EEFFE110D2E6EFF0E0A0EEB0E06BD058
:10130000F4D40895E3E0F1E0AAD2E881F981A2D211
:1013100098D3FF27EDE0ADE7B0E0ECD4E7E0F1E0F3
:10132000D080EE24FF240027B9D2E9D2EDE7F0E027
:1013300091D200D3FF27EDE0ADE7B0E0DBD48FEB37
:1013400011E06DD0E8ECFFE155D05A924A92EDE7FA
:10135000F0E0A42DB52DCED484E012D085DF229606
:1013600084E00AD08FEB11E05AD0A0EEB0E03CD080
:10137000EAEEFFE13FD00895481A8827580A0895F9
:10138000480E8827581E0895ED91FC913196FC93E4
:10139000EE93089504D0B5D100FC0CD0089500243C
:1013A000E89457FF02C009D0689400F80BD010F8F9
:1013B0000124089502D009D00895509540954F5FBB
:1013C0005F4F0895E89417FF0895009510950F5FFB
:1013D0001F4F689408958F938D918823E9F7119793
:1013E0008F910895A0EEB2E08D91882311F064D022
:1013F000FBCF089583D3802D11F05ED0FBCF0895ED
:1014000081E060D014D080E85DC08FE7213039F0F2
:101410008FEB223021F08FE8233009F08FEC810F21
:1014200051C088EE93E07FD03197D9F7089583E0DB
:10143000992779C08AEF90E076D0A09AA19AA29AD3
:10144000A39AA49AA59AAD9885E090E06CD0AC9848
:10145000A898A998AA9AAB9AAC9AEF93FF93E4EC58
:10146000F0E055D0FF91EF91AC985AD0AC9AEF9341
:10147000FF93E4ECF0E04BD0FF91EF91AC9850D0AB
:10148000AC9AEF93FF93E4ECF0E041D0FF91EF9141
:10149000AC9846D0AB98AC9AEF93FF93E4ECF0E0B5
:1014A00036D0FF91EF91AC983BD088E20BD08EE024
:1014B00009D086E007D00895AD9A829505D004D072
:1014C0002FD00895AD98F9CF859510F4AB9A01C04F
:1014D000AB98859510F4AA9A01C0AA98859510F446
:1014E000A99A01C0A998859510F4A89A01C0A89856
:1014F000AC9AEF93FF93E4ECF0E009D0FF91EF9109
:10150000AC98089504231523262337230895319793
:10151000F1F70895689462F80895E89462F80895E0
:1015200081E090E000C0EF93FF93EE27E82BE92BDA
:1015300031F0E0EDF7E03197F1F70197D1F7FF9146
:10154000EF9108958DE207FD8D938F2D881F802FD9
:10155000881F8F57082F6894F7F8802F87FF15C0D2
:1015600080958395082F80E38D938EE28D93802F55
:10157000815228F080E38D9399279C930895442706
:101580000A95802F09F192D01FC0805230F09EE45E
:101590009D9381E48D939D93EFCF4427DF92EF924B
:1015A000FF920F938FE1801B11F0082F7FD085D021
:1015B0009EE29D930F91FF90EF90DF90442703955B
:1015C000003209F4D7CF27D03F93ECE4F6E138E1BD
:1015D0002F2D1E2D0D2DFF24EE24DD244427000F7A
:1015E000111F221F88F42F923F9288D2102C86D28E
:1015F000202C84D2302C82D23197410DD21CE31C96
:10160000F01C3F902F9001C0339631963A9539F7F0
:101610003F9107D0B3CFDD0CEE1CFF1C0A95D9F724
:101620000895002719E058D08F93802B11F003956F
:1016300001C08F911A95B9F7802F882309F49ACFAA
:101640008F91805D8D930A95D9F796CF0065CD1D5A
:1016500080B2E60E40597307A0ACB90350D6DC0146
:10166000286BEE0094357700CA9A3B0065CD1D00CB
:10167000B2E60E0059730700ACB90300D6DC0100D6
:101680006BEE0000357700009A3B0000CD1D000096
:10169000E60E000073070000B9030000DC01000043
:1016A000EE000000770000003B000000F694E79495
:1016B000D79447950A95D1F7089500270DD08F93B9
:1016C00003958F2D8E298D29842BC1F78F91805DF5
:1016D0008D930A95D9F750CF1F930F93002710E2EF
:1016E000440FDD1CEE1CFF1C001F802F9AE0890BAD
:1016F00010F0082F43951A9599F7802F0F911F919D
:1017000008950F92B801469F8001479F100D569F84
:10171000100D0F900895F2D10D920020E1F7089579
:10172000903029F08C91880F9A95E9F78C93089561
:10173000903029F08C9186959A95E9F78C930895CD
:10174000903041F00D911C91169507959A95E1F70F
:101750001C930E930895903071F00D911D912D9171
:101760003C9136952795179507959A95D1F73C9317
:101770002E931E930E93089599910027A90FB01FE1
:101780001197492F4A955E2F6F2FE89411274395A3
:10179000203019F0C895802D01C080818823B9F0D0
:1017A0007C917723A1F0781739F40EF0042F13956C
:1017B000689411963196EBCF112321F0411BA11BA8
:1017C0001127B10BE894E52FF62F1196E0CF88236F
:1017D00011F00027089508953DD0992711278F2DE6
:1017E000880F80E8F82A802F881F08F41FEF41F047
:1017F0008F57082F07FD04C0003240F08FEF01C063
:101800008827982FD82EE82EF82E09C08FE1801B4C
:10181000082FF694E794D79497950A95D1F711235A
:1018200051F09095D094E094F09481E0980F88273F
:10183000D81EE81EF81E0F2DFE2CED2CD92E089573
:10184000D094E094F09491E0D90E9927E91EF91E06
:1018500010950895D190E190F19001910895219112
:101860003191419151910895102F90E8FF0C001F84
:101870000927990FF7941078652F90E8440F551FAA
:101880005927990F4795607800380895FF0C90E824
:101890009027110F9795F794092F0895102FBD2CBD
:1018A000DE2CEF2CF02E11234AF4B094D094E09467
:1018B000F0949FEFB91AD90AE90AF90A0EE1FF205C
:1018C00039F4FE2CED2CDB2CBB240850C2F766C08B
:1018D00032F00A95BB0CDD1CEE1CFF1CF9CF01D0C9
:1018E000D5CFB7FE089590E8B91611F4D0FE08954B
:1018F0009FEFD91AE90AF90A09F403950895502FC0
:101900002D2D3E2D4F2D612F08952DEC3CEC4CECF0
:101910005DE366270FC09EDFF2DFDD24EE2490E852
:10192000F92E0FE307C09BDF05C02227332740E2D3
:1019300051E46627552351F1002381F195DF71F1C0
:101940001627005850580894050B18F407FD03C0DB
:1019500025C007FD23C0469537952795F694E79453
:10196000D79422D0FF202AF0DD0CEE1CFF1C015082
:1019700073F09D2D969548F0DD203AF4EE202AF480
:1019800091E0D90E9927E91EF91E80CF07C09FE785
:10199000092FF92A9FEFD92EE92E0895DD24EE2490
:1019A000FF240027112708959F929924AA24BB247D
:1019B00088E1D216E306F40628F0D21AE30AF40A04
:1019C000089401C08894991CAA1CBB1CDD0CEE1C59
:1019D000FF1C8A9571F7D92CEA2CFB2C9F90089557
:1019E00043DFE1F25038D1F21627005850580894DE
:1019F000051F12F418F4CBCF08F0D0CF0AD0FF2087
:101A00002AF0BB0CDD1CEE1CFF1C40CF0F5FFBF16E
:101A10003DCF9F929924AA24BB24992788E1990C51
:101A2000AA1CBB1CDD1CEE1CFF1C30F4920EA31E76
:101A3000B41ED91EE91EF91E8A9589F79F90089554
:101A40000EDF12DF503829F090E869270CC00AF049
:101A500045D01CCF5FE322273327442701C0FFDE98
:101A600003DF5038B1F3003899F3902F951B8BF3B7
:101A700012F434D0FACF983118F0222733274427B4
:101A8000983028F0232F342F44279850F9CF9923EA
:101A900029F04695379527959A95D9F7912F96274E
:101AA00042F014D0B0F6F794E794D7940F5F8BF61A
:101AB0006ECF10D051F008F4C3DEFF2052F2DD0CDF
:101AC000EE1CFF1C0150CBF762CF68CFD20EE31E95
:101AD000F41E0895D21AE30AF40A0895DF92EF92F1
:101AE000FF920F931F93D22EE32EF42E052F162F65
:101AF0006F915F914F913F912F910895C8953196C5
:101B000000200895FBDFD02CF9DFE02CF7DFF02C6C
:101B1000F5DF002D0895F2DF202DF0DF302DEEDF10
:101B2000402DECDF502D089507FB00680EF40F7771
:101B300057FB50680EF45F7707FD02C057FF05C0E2
:101B4000D216E306F406050708952D153E054F0548
:101B50005007089591E005C092E003C094E001C0F1
:101B600098E0CCDF0D929A95E1F7089599278D9131
:101B700093958823E1F7939511968C9311978E9105
:101B80009A95D1F70895EA2FFB2F00244C918D915F
:101B900003948E32E1F711248D9113948823E1F799
:101BA0001A94101640F41197202F2119239580E3E1
:101BB0008D932A95E9F7113039F59927AE2FBF2F6C
:101BC000A00DB91FA00FB91F8C919C93853308F409
:101BD00021C031E08E918E32E9F38D3241F0830FD6
:101BE0008A3319F480E331E001C033278C93AE17B8
:101BF00089F7332341F0AE2FBF2FB8DF81E34D3299
:101C000009F43196808308958827E00DF81FE00FCE
:101C1000F81F80830895000F111F221F331F08959E
:101C200000951095209530950F5F1F4F2F4F3F4F18
:101C30000895019110810EC001911191219130817F
:101C40000BC00191108117FF05C03FEF2FEF04C0BB
:101C5000008111272227332737FF03C0E1DF8DE200
:101C60008D93CF93DF93CF92DF92EF92AA24BB2480
:101C7000CC24DD24EE2440E2CAE0DD2755E093E3E6
:101C80008881890F87FD9F7083FD907F891B8993D1
:101C90005A95A9F7C0DFAA1CBB1CCC1CDD1CEE1C8E
:101CA0004A9551F7E894EFE0FF2782910ED0EB3090
:101CB000E0F71EF068948A2D0CD088278D93EF9062
:101CC000DF90CF90DF91CF910895982F829501D02A
:101CD000892F8F70805D26F0803309F40895689411
:101CE0008D93089588278D93089581918D938823EE
:101CF000E1F7089594E081918D939A95E1F7089525
:101D000081918D930A9519F08823D1F70895EACF30
:101D1000E199FECFEEBBFFBB3196089591E001C083
:101D200092E07B3751F47FB7F894F2DF8D918DBB51
:101D3000E29AE19A9A95C9F77FBF7727089591E0D3
:101D400001C092E0E5DFE09A8DB38D939A95D1F7CB
:101D500008958FEF83959D919923E1F708957ADD9A
:101D60000F77089577DD80DD0395AAF087E1DD0C1C
:101D7000EE1CFF1C8A9589F00A95CAF7FF205AF0DD
:101D800000240D280E280F28002039F00A95DD0CBC
:101D9000EE1CFF1CDAF70A9579CD00CE5BDD80E002
:101DA00003C058DD802F8078882321F0DF92EF92E6
:101DB000FF920F938F9358DD802F839512F4EEDD01
:101DC0001BC080958A95885E0AF415C088501AF465
:101DD0000CD0D92210C0DD2488501AF406D0E92294
:101DE0000AC0EE2402D0F92206C09FEF8770990F37
:101DF0008A95EAF708954ADD8F918823D9F35F9198
:101E00004F913F912F910F938FDE0F9199F390F3A4
:101E100012D0506825CE1EDD802FFF0C001F090F49
:101E200030F00F3F21F0881F0795F7940895AFDD3C
:101E30008078082B08955FE340E833272227089530
:101E4000C198C298B998BA980895BA9AB99803D027
:101E5000BA9801D0B99AEF93FF93E6E0F0E057DB30
:101E6000FF91EF910895BA9AB99AF5DFBA98B29BAB
:101E7000FECFF1DFB998EFCF0894111F01C0110F09
:101E800069F0BA9A18F40000B99802C0B99A00C073
:101E9000E2DFBA98B29BFECFDEDFF1CFBA9AB998F3
:101EA000DADFBA98B29BFECFE894B199689462F8F1
:101EB000D2CFACC5273717B7D1386F12833A0AD7BC
:101EC000233CCDCCCC3D0000803F000020410000F1
:101ED0000000000080400000004100008041000040
:101EE00000420000804200002043000060400030BB
:101EF000B14500909745000088410000684100000E
:101F0000E5420000E442CDCCCC3ECDCCCCBE7370DB
:101F100036667265205349353730207631340000FB
:101F2000687474703A2F2F6C782D6E65742E706CF7
:101F300000003130487A0000313030480000202065
:101F4000316B00002031306B00003130306B00000D
:101F50002020314D0000435775004357640055530E
:101F600042004C5342004F4600004F4E2000463185
:101F7000000046320000463300004634000046357B
:101F800000005345545550004678203D2000466FD0
:101F900066203D200000444956203D20000020528C
:101FA00049543A00202000005249543A000041436D
:101FB00054494F4E000045584954000053455420A1
:101FC00046782D74616C00002020202020202020E5
:101FD0002020200053455420466F6600534554206E
:0C1FE00044002020202020002E0048009B
:00000001FF
